:10000000803102288731F52F8631FA2E8731022F71
:0C00100087310A2F8731122F87311A2FF9
:10081E00640080010131890B102C00342000A81BCC
:10082E001A2C290808000030080014303D009100F1
:10083E0008308E001130920008002000D6010830DA
:10084E00A1008830F0007008A000A401080020006C
:10085E00AC1B08000830F3007308AD002C30843157
:10086E00522408002000A81B08000830F30073086B
:10087E00A9002830843152240800FC302100990050
:10088E00903027009B00043021008E0022008E0144
:10089E002000D2010800F2007208F000F101700889
:1008AE0020008600710887000109403988388100D0
:1008BE00080084314424843184311C248431200086
:1008CE00121D6C2C85310225843184318F248431A4
:1008DE00662C8030F00070082000C80000300E1921
:1008EE000130C90000308E190130CA000330F0000B
:1008FE007008F10008307102031808007108483EB4
:10090E008600870181010130F0007008F107812C0B
:10091E003D001608031D8E18B52C84311524843124
:10092E00003A0319B52C803020004006031DA22C7E
:10093E00843170248431813020004006031DAF2C99
:10094E008E1DAB2C8E11AC2C8E15843170248431FF
:10095E0084313924843184312E24843120000E0CCC
:10096E00890C013952060319080084317024843130
:10097E0084312E24003020000E190130D2000800E0
:10098E0008307D02031CCF2C0830F2000030D52C2D
:10099E007D08F000F1017008F2007108F300720892
:1009AE00F0007008F5007508F00070082000A50032
:1009BE007508FD025730F0007008D400F401750878
:1009CE0074020318080050088400510885000008BE
:1009DE00F000540886008701700881000130D007AE
:1009EE000030D13D0130F0007008D4070130F00026
:1009FE007008F407E62C3D001019121D092D8E10FB
:100A0E00121110118E1C0F2D9001200012110800D2
:100A1E00101C322D930190019F3097007B30920075
:100A2E0016309800901D1D2D9011192D0E120230AA
:100A3E00203E860087013730C03F2030C13F203036
:100A4E002000A7003730A6008431242485312000F1
:100A5E00D5013D001010101E372D12158E141012D8
:100A6E00101B1013901E432D181C422D843124246C
:100A7E0085313D0018109012901C472D9010930157
:100A8E00901D4D2D85319F253D0090112000121196
:100A9E000800A230F2007208F60070088400710897
:100AAE0085000008F200F3017208F7007308F800E1
:100ABE00770878040319922D0130F0070030F13DCC
:100ACE00F71F862D700884007108850000083F39D5
:100ADE00F200F3013F307705F40000307805F500A1
:100AEE000630F435F50D890B782D72087404F70075
:100AFE0073087504F8000130F0070030F13D7608F8
:100B0E00860087017708C03F7808C13F0230F200A7
:100B1E007208F607542DA030FF3A013E7607F20018
:100B2E0072082100A0000330F2007208A100080034
:100B3E002D2E3C3020002005FC0034307C06031D99
:100B4E00E52D7F30FC007C08A4057F30FC007C087E
:100B5E00A005D6018631372685313D000E1E0800D0
:100B6E002000D71FD52D7D085D020318C22D5D080C
:100B7E00FC007C08FD008431C72485310230FC0066
:100B8E007C082000D6000830A1008030FC007C08D4
:100B9E00A000C830FC007C08A400E22DD601D60AC5
:100BAE00A501C830FC007C08A4000830A100C830A4
:100BBE00FC007C08A0003D000E1208002000560329
:100BCE00031D2A2E2108FC007C08E6006608FC00A6
:100BDE007C08FD075730D0000030D100E5016608D3
:100BEE0065020318122E5008840051088500000873
:100BFE00FC005408860087017C0881000130D00774
:100C0E000030D13D0130FC007C08D4070130FC00DF
:100C1E007C08E507F62D2030843152240800200090
:100C2E00530803191F2E53083D0096002000D301D0
:100C3E0002305606031D2A2E8431C72485312430F6
:100C4E008431522408008431242408003D000F080A
:100C5E00003A0319A02D043A0319162E362E080059
:100C6E00FD012000D71FD02F2100A001A101A0302F
:100C7E002000D0000030D100D02F5903031DE72FE4
:100C8E0002305805F9005508FD397904FA007A0842
:100C9E00D50008005908F9007908D3000800023081
:100CAE0059020318E72F5908F9007908D50055089D
:100CBE000319E72F1E303D0099009A000830F90005
:100CCE0079082000A9002030AB002030AA0088301F
:100CDE00F9007908A8002030AF002830AE0040306F
:100CEE00F9007908AC004030F9007908B1002130E4
:100CFE00B3008030B2008830F9007908B00021309E
:100D0E00B7000030B6004030F9007908B400080092
:100D1E005808013A0319442E023A0319442E063A92
:100D2E000319512E0C3A0319562EE72FE72F5808A8
:100D3E000B3A0319F42FE72FE72F5B08F900790818
:100D4E00E4006408F9000130F935890BAB2E640814
:100D5E00FA000730FA36890BB12E7A087904FB00B7
:100D6E007B08E4005908031DE72F063064020318C0
:100D7E00E72FD818D02E6418C92E8830E100003025
:100D8E00E200CB2EE101E2016208E0006108DF0023
:100D9E00D42E8430DF000030E0005F08F9006408D4
:100DAE00FA000130FA35FF3E031DD92E7A35203E6A
:100DBE00860087017908810008005808013A031956
:100DCE00A42E023A0319A42EE72FE72F9A30D00053
:100DDE008830512F0030D0008830D1004030F900DB
:100DEE007908FD000800CF30F0008830F100853121
:100DFE0050258631522FCB30F0008830F1008531EE
:100E0E0050258631522F8730F0008830F100853121
:100E1E0050258631522FBD30F0008830F1008531DB
:100E2E0050258631522FAC30F0008830F1008531DC
:100E3E0050258631522F20005908840005300402B7
:100E4E000318E72F80310435043E8200E72F5A083D
:100E5E00013A0319ED2E033A0319F12E013A031943
:100E6E00222FE72FE72F55080139F90079082100C5
:100E7E00A000772F20005808003A0319AF2F063A2A
:100E8E0003192E2F0E3A03193A2FE72FE72F1230A0
:100E9E00D0008830D1002000500884005108850011
:100EAE000008F9007908FD0008004030D0008830B5
:100EBE00D1002F30F9007908FD0008005A08213AB8
:100ECE0003194E2F033A03195C2FE72FE72F58080B
:100EDE00063A0319652F0C3A0319772FE72FE72FE0
:100EEE00FD01FD0A0800200058080A3A0319772F61
:100EFE00E72FE72F5B08003A03196E2F013A03190B
:100F0E007A2FE72FE72F5B08F9007908E3006308D3
:100F1E00F9000130F935890B912F6308FA0007307B
:100F2E00FA36890B972F7A087904FB007B08E300C9
:100F3E006308F9000130F935FF3E031DA22F793504
:100F4E00203E86008701011DAF2F2100A001A00ABF
:100F5E000230F9007908FD00080020005808003A18
:100F6E0003198A2FE72FE72F6F30D0008830D1007A
:100F7E001830F9007908FD0008005808073A0319DF
:100F8E00BB2FE72FE72F5B08013A0319C42FE72F7A
:100F9E00E72F5708003A03198F2E013A03199E2E98
:100FAE00033A0319E42E823A0319412F013A031929
:100FBE00812F033A0319B42F233A0319CA2FE72FAF
:100FCE0008302000A1008430F9007908A000843098
:100FDE00F9007908A4003D000E120800FD01503002
:100FEE008400003085000F3084310F2420008431BE
:100FFE00602C09340234403400340234013400349D
:10100E00A034193409340434003400340234033467
:10101E0000340034033409342134113401340034E3
:10102E00013422342F3400340734053401340334B0
:10103E000834003401340734053481340334083461
:10104E000034013409340434013400340234FE34E3
:10105E00033400340434073405340234023440348B
:10106E000034003407340534823402344034003402
:10107E0000340634A034FF3409340134A134013471
:10108E0009340134153400342634FF3400347534F9
:10109E00083495340834813402340934013415345B
:1010AE0000342634FF340034753408349534083453
:1010BE009134023409340234153400342634FF34AA
:1010CE0000347534083495340834B1340234C034E5
:1010DE000134003400340134003400340034003460
:1010EE000034003400340034003400340034003452
:1010FE000034003400340034003400340034003442
:10110E005034433453343534303430342034553441
:10111E005334423420344134643461347034743482
:10112E006534723400341234013400340234003425
:10113E00003400340834D8340434A5340134013476
:10114E000034013402340034013455345334423403
:10115E0054344D344334203449346E34743465344D
:10116E00723466346134633465340034483449343F
:10117E004434203449346E347434653472346634F5
:10118E00613463346534003468342334733400348A
:06119E00D0348934003456
:020000040001F9
:04000E00E4CFCFFF6D
:00000001FF
